S10E80008EFFBFBD94A74FCE9AEB8CFF
S111800B9B182705A7000820F6CE9AE718CE8A
S11180199AE98C9AE9270AE60018E70008188D
S11180270820F1CC0000270CC39B183736CC80
S10E80359B18BD88BF38BD990A20FECF
S11180400F18CE103C181C000B18CE103C1864
S110804E1D0004CC0000FD9B0CCC0000FDC7
S111805B9B0ECC0000FD9B10CC0000FD9B1280
S1108069CC0000FD9B14CC0000FD9B16CC48
S11180760000FD101618CE1022181C00800EFB
S111808439BD86BA46EC08ED02FC9B0CE30203
S1118092ED041AA302250AFC9B0C1AA3042574
S11180A0F8200DFC9B0C26FBFC9B0C1AA30481
S11080AE25F88FC300068F3538183839FCCB
S11180BB1016C307D0FD1016FC9B16C300015F
S11080C9FD9B161A8303E8260FCC0000FD72
S10F80D69B16FC9B14C30001FD9B14FCD2
S11180E29B141A83003C260FCC0000FD9B1457
S11180F0FC9B12C30001FD9B12FC9B121A8321
S11180FE003C260FCC0000FD9B12FC9B10C31F
S111810C0001FD9B10FC9B101A830018260F27
S110811ACC0000FD9B10FC9B0EC30001FD7A
S11081279B0EFC9B0CC30001FD9B0C18CEAD
S10A81341023181D007F3B1E
S109FFD69813981498151D
S109FFDC9816981781EA53
S109FFE282E4981898EB7C
S109FFE880BA9819981A72
S109FFEE981B981C981DED
S109FFF4981E981F9820DE
S109FFFA9821982280000A
S111813B18CE1039181C00803937363C3C3001
S1118149EF00EC04F71030F61030C480C18053
S110815726F7F610314F080835381838396E
S11081640F18CE1020181D0003CC0000FDE4
S11181719AF2CC0000FD9AF0CC0000FD101E26
S111817F7F9AEDCC0000FD9AEEC680F79AEBD5
S111818DC608F79AEC18CE1026181C008818A5
S111819BCE1022181C00080E3937363C3C303A
S11181A9EF00EC081A8307D02C22EC08271EE6
S11181B7EC042610EC0805050540508200C3B8
S11181C50BB8ED08200AEC08050505C30BB83D
S11181D3ED08EC045818CE9AF0183AEC08188F
S11181E1ED0008083538183839BD86BA0A187A
S11181EFCE9AED181D00FCF69AED4F5D2A01A4
S11181FD43ED044756E706EC048400C401E792
S111820B07E6064F5D2A014305C39AF0188F5B
S111821918EC00ED0826126D07260EFC101E50
S1118227C34E20FD101E7C9AED20336D0727F8
S111823512CC4E20B39AEEED02FC101EE302B2
S1118243FD101E2008FC101EE308FD101EE6B0
S1118251064F5D2A0143C39AEB188FF6100006
S111825F18E800F71000EC08FD9AEE7C9AED8A
S111826DF69AEDC10426037F9AED18CE102375
S10F827B181D00F78FC3000A8F35383B34
S11182870FCC82E4FDFFE2CC0000FD9AFECC99
S11182950000FD9AFCCC0000FD9AFACC00001B
S11182A3FD101C7F9AF7CC0000FD9AF8C6105F
S11182B1F79AF4C620F79AF5C640F79AF61825
S11182BFCE1022181C00100E3937363C3C300D
S11182CDEF00EC045818CE9AFA183AEC081890
S11182DBED0008083538183839BD86BA0A187F
S11182E9CE9AF7181D00F8F69AF74F5D2A0199
S11182F743ED044756E706EC048400C401E797
S111830507E6064F5D2A014305C39AFA188F56
S111831318EC00ED0826126D07260EFC101C57
S1118321C34E20FD101C7C9AF720336D0727F5
S111832F12CC4E20B39AF8ED02FC101CE302AF
S111833DFD101C2008FC101CE308FD101CE6BB
S111834B064F5D2A0143C39AF4188FF6100002
S111835918E800F71000EC08FD9AF87C9AF77B
S1118367F69AF7C10626037F9AF718CE102364
S10F8375181D00EF8FC3000A8F35383B41
S111838118CE1028181D0020C6B0F7102BC609
S111838F0CF7102D39BD86BA04CC0000ED02A7
S111839D200AF6102E4F8400C420ED02EC02DC
S11183AB27F2F6102F4F8400C47F080808083C
S11183B9353839BD86BA44CC0000ED02200AE6
S11183C7F6102E4F8400C480ED02EC0227F263
S11183D5EC06F7102F08080808353818383958
S11183E3BD86BA46CC0000ED04CC0000ED02CD
S11183F1204AEC04E308188F18E600C15C264D
S11183FF25EC04C30001E308188F18E600C142
S110840D6E2615CC000DBD83BCCC000CBD4B
S111841A83BCEC04C30002ED042018EC04E360
S111842808188F18E6004F5D2A0143BD83BC7F
S1118436EC04C30001ED04EC04E308188F18F5
S11184446D0026AB8FC300068F35381838390B
S1118452BD86BA46CC0000ED02EC082C0ECC20
S1118460002DBD83BCEC0840508200ED08CC1A
S111846E0000ED04200EEC08832710ED08EC4E
S111847C04C30001ED04EC081A83270F2EEA56
S110848AEC042F0DEC04C30030BD83BCCC0A
S11184970001ED02CC0000ED04200EEC088381
S11184A503E8ED08EC04C30001ED04EC081A32
S11084B38303E72EEAEC042E08EC021A8382
S11084C00001260DEC04C30030BD83BCCCCC
S11184CD0001ED02CC0000ED04200EEC08834B
S11184DB0064ED08EC04C30001ED04EC081A83
S11084E98300632EEAEC042E08EC021A83D3
S11084F60001260DEC04C30030BD83BCCC96
S11185030001ED02CC0000ED04200EEC088314
S1118511000AED08EC04C30001ED04EC081AA6
S110851F8300092EEAEC042E08EC021A83F6
S111852C00012608EC04C30030BD83BCEC083B
S111853AC30030BD83BC8FC300068F353818D4
S1108548383937363C3C30EF00CC0020BD04
S111855583BCEC04BD8452CC000DBD83BCCCB1
S1108563000ABD83BC08083538183839BD3E
S111857086BA0ACC0000ED04BD8394ED08BD6C
S111857E83BCEC081A83002D260DCC0001ED01
S110858C04BD8394ED08BD83BCEC081A8384
S1118599002B260DCC0000ED04BD8394ED08EC
S11085A7BD83BCCC0000ED062023EC08834E
S11185B40030ED08EC060505053736EC06052B
S11185C2ED023233E302E308ED06BD8394EDCF
S11185D008BD83BCEC081A8300302D08EC08AB
S11085DE1A8300392FCDCC000DBD83BCCC19
S11185EB000ABD83BCEC041A8300012608ECD0
S11185F906405082002002EC068FC3000A8F59
S1068607353839C6
S111860A3C183C38028F38393C364D2A054363
S111861853C30001183C3818308C00002A08A7
S11186268F43538F08186300028F186D002ACB
S10C8634054353C3000131383938
S111863D3C183C380238393C364D2A0543536C
S111864BC30001183C388C00002A058F4353ED
S11186598F0802306D002A054353C30001311F
S105866738399C
S11186693C183C37363C3C30CC0000ED00A6FB
S111867705E6073DED02A605E6063DE301ED2E
S111868501A604E6073DE301ED016900A60429
S1118693E6063DE300ED00183832333838387F
S10486A1399B
S11186A21A83000027113718E600E70033831F
S10D86B00001270508180820EF391F
S11186BA1838181F00400237363C3018E6000E
S11186C84FC43F37368F30A3008F35EF0018B4
S11186D61F0080043C3C3C3C186E01183037F9
S11186E436188F183018EE0218EB00890018B3
S11186F23018EE02188FC3000118ED00323369
S1068700183539EC
S111870318CE102E181F0020F7F6102F4F3935
S111871137363C3C30EF00E605C10A2606CCA4
S111871F000DBD871118CE102E181F0080F714
S111872DE605F7102FE6054F5D2A0143080804
S108873B35381838393F
S111874037363C3C30EF00EC04F7102BC60C2F
S10D874EF7102D08083538183839E3
S1118758BD86BA56EC1C2608CC87E4ED127ED2
S111876687C86F11EC00C30011ED1220511AE8
S1118774EE1EEC1CBD863DED141A83000A2C8B
S110878216EC12C3FFFFED05ED12EC14C35D
S111878F00301AEE0518E7002021EC1E1A83B4
S111879D00102619EC12C3FFFFED03ED12ECE1
S11187AB14C387D3188F18E6001AEE0318E7DC
S11187B9001AEE1EEC1CBD860AED1CEC1C26FC
S11187C7ABEC123736EC18BD940F18388FC384
S11187D500168F3538183839616263646566A2
S10687E30030005F
S11187E6BD86BAE4EC00C3002A188FBD88F8E3
S11087F418CE88BBBD891EBD8D862608CC1D
S111880188B9ED207E889D6F1FEC00C3001F18
S110880FED207E8884EC00C3002A188FBD84
S10E881C88F8EC2EBD89A0BD8BF1BDD7
S110882789DFED221A83000A2C16EC20C311
S1118834FFFFED04ED20EC22C300301AEE0429
S111884218E7002021EC2E1A8300102619ECF2
S111885020C3FFFFED02ED20EC22C388A81820
S110885E8F18E6001AEE0218E700EC00C3C4
S110886B002A188FBD88F8EC2EBD89A0BD31
S11188788BB2EC00C3002A188FBD8935EC00CA
S1108886C3002A188FBD88F818CE88BBBD2A
S1118893891EBD8D8627037E8814EC2037369F
S11188A1EC26BD940F18388FC300248F353891
S11188AF1838396162636465660030000000A9
S10588BD0000B5
S11188BFBD86BA46EC08ED041AEE04FC9B00DC
S11188CD18ED00EC04FD9B00EC08C30006ED62
S11188DB02EC0CA3021AEE0418ED041AEE04CB
S11188E9EC0C18ED028FC300068F35381838DA
S10488F73943
S11188F837368F8300088F18EC00ED0418EC5F
S111890602ED06C6083A323339373618EC0053
S1118914ED0418EC02ED0632333937368F834A
S111892200088F18EC00ED0018EC02ED02C600
S1118930083A32333937368F8300088FEC044F
S111893E18ED00EC0618ED02C6083A32333983
S111894C3736EC0418ED00EC0618ED02323359
S111895A3937368F8300088FEC0018ED00ECDF
S11189680218ED02C6083A32333937368F83CF
S111897600088FEC04ED00EC06ED02C6083A92
S111898432333937368F8300088F6F046F0546
S11189923233ED062C0463046305C6083A393B
S11189A037368F8300088F6F006F013233ED7E
S11189AE022C0463006301C6083A3937368F81
S11189BC8300088F3233ED066F046F05C60882
S11189CA3A3937368F8300088F3233ED026F4F
S11189D8006F01C6083A398F8300088FEC0641
S11189E637C6083A33393736183018EE02EC2B
S11189F40018E300188F18EC00830004188F9D
S1118A02BD893532331838186E02183C18300E
S1118A1018EE02183C183018EE02183C37C657
S1118A1E051830183ABD893532183839183C1D
S1118A2C183018EE02183C183018EE02183CF0
S1118A3A37C6051830183ABD895B3318383931
S1118A48183C3736C6061830183ABD88F818A0
S1118A563018EC0418ED083233183831313181
S1108A643139183C3736C6061830183ABDB3
S1118A71891E183018EC0418ED08323318383A
S1088A7F3131313139F1
S1118A8437368F8300088FEC06E302ED06EC14
S1118A9204E901A900ED04C6083A323339376D
S1118AA0368F8300088FEC06A302ED06EC046B
S1118AAEE201A200ED04C6083A32333937362D
S1118ABCEC06A302ED06EC04E201A200ED04B8
S1118ACA3233393736183C8F8300088F3C3C1A
S1118AD8EC061AEE02BD8669183C1830180828
S1118AE6180818ED02EC061AEE00BD8669377A
S1118AF436EC041AEE02BD8669183018E30051
S1118B021838183018E30018381830ED04182D
S1118B10EC02ED0618381838C6083A18383248
S1118B1E3339CC000018ED0018ED02C62037E4
S1118B2C680769066905690418690318690277
S1118B3A18690118690018EC001AA300270737
S1118B48251E18EC02200818EC021AA30225C0
S1118B5611A30218ED0218EC00E201A20018AF
S1118B64ED006C07335A26BF39EC04E801A873
S1118B72002A04C6012002C60037EC042A03C0
S1118B80BD8D4BEC002A03BD8D60BD8B2033F0
S1108B8E5D2703BD8D4B393736183C8F83AE
S1118B9B00088F183C183C18308DC718381885
S1118BA938C6083A18383233393736183C8F3C
S1118BB78300088F183C183C1830BD8B201822
S1118BC5381838C6083A18383233393736189B
S1108BD33C8F8300088F183C183C1830BDFF
S1118BE08B6DBD890F18381838C6083A18383E
S1118BEE3233393736183C8F8300088F183C19
S1118BFC183C1830BD8B20BD890F183818386E
S1118C0AC6083A183832333937368F830008DB
S1118C188FE603C41F5D270B68076906690514
S1108C2669045A20F2C6083A3233398F83AC
S1118C3300088FC41F5D270B680769066905DA
S1108C4169045A20F2C6083A3937368F8389
S1118C4E00088FE603C41F5D270B670466054C
S1118C5C660666075A20F2C6083A3233398F8C
S1118C6A8300088FC41F5D270B670466056630
S1118C780666075A20F2C6083A3937368F834B
S1118C8600088FE603C41F5D270B6404660517
S1118C94660666075A20F2C6083A3233398F54
S1118CA28300088FC41F5D270B6404660566FB
S1118CB00666075A20F2C6083A3937368F8313
S1118CBE00088FEC04E401A400ED04EC06E4CD
S1118CCC03A402ED06C6083A32333937368F58
S1118CDA8300088FEC04EA01AA00ED04EC0606
S1118CE8EA03AA02ED06C6083A3233393736DB
S1118CF68F8300088FEC04E801A800ED04EC65
S1118D0406E803A802ED06C6083A32333937F2
S1118D12368F8300088FCC0000A306ED06CC3C
S1118D200000E205A204ED04C6083A3233391D
S1118D2E37368F8300088FCC0000A302ED02BD
S1118D3CCC0000E201A200ED00C6083A32337A
S1118D4A393736CC0000A306ED06CC0000E25B
S1118D5805A204ED043233393736CC0000A3F3
S1118D6602ED02CC0000E201A200ED00323367
S1118D74398F8300088F630563046307630669
S1118D82C6083A393736183C8F8300088F181C
S1118D903C183C1830BD894CBD8ABA0784F0EB
S1118D9E36EC042608EC062604328A0436EC71
S1118DAC0427062A04328A0836EC00CDA30000
S1118DBA2209250BEC02CDA3022304328A0108
S1118DC836EC042B0F18EC001A83000024175D
S1118DD6EC002B13200D18EC002B0CEC001AF3
S1118DE48300002404328A0236C6083A32069E
S10C8DF2183818381838323339E6
S1118DFBBD86BAF8CC0000ED2F7E93B71AEEB9
S1118E094018E600C12527211AEE4018E600A5
S1118E174F5D2A01433736EC3A1AEE3E18AD91
S1118E25001838EC2FC30001ED2F7E93B0EC43
S1118E3300C30010ED29CC0000ED34CC00008B
S1118E41ED32CC0000ED2DC620E731EC40C32D
S1118E4F0001ED40CC0000ED361AEE4018E6AE
S1118E5D004F5D2A0143ED081A830020274CC4
S1118E6BEC081A8300232722EC081A83002047
S1118E792D54EC081A83002B2726EC081A83CC
S1118E87002D2714EC081A8300302732203AFD
S1118E95EC348A00CA01ED342035EC348A0036
S1118EA3CA04ED34202BEC348A00CA08ED34E6
S1118EB1C62BE731201DEC348A00CA08ED34CC
S1118EBFC620E731200FEC348A00CA10ED34CF
S1118ECD2005CC0001ED36EC362702200AEC1D
S1118EDB40C30001ED407E8E581AEE4018E6AA
S1118EE9004F5D2A0143BD96E11A8300002765
S1108EF724EC40BD94DDED322007EC40C3B7
S1118F040001ED401AEE4018E6004F5D2A0110
S1118F1243BD96E11A83000026E51AEE4018CE
S1118F20E600C12E2629EC40C30001ED40BD41
S1118F2E94DDED2D2007EC40C30001ED401A48
S1118F3CEE4018E6004F5D2A0143BD96E11A8F
S1118F4A83000026E51AEE4018E600C16C26EE
S1118F580FEC40C30001ED40EC348A00CA0265
S1118F66ED341AEE4018E6004F5D2A0143ED8B
S1118F74081A83006F26037E90B1EC081A835E
S1108F82006F2E20EC081A83006326037E86
S1118F8F921FEC081A8300642751EC081A8321
S1108F9D006626037E93A82023EC081A83A7
S1118FAA007326037E9246EC081A8300752697
S1108FB8037E90B1EC081A83007826037E36
S1118FC590B120001AEE4018E6004F5D2A011C
S1118FD3433736EC3A1AEE3E18AD001838EC6F
S1118FE12FC30001ED2F7E93B0EC348400C446
S1108FEF021A83000026037E906EEC42C33C
S1118FFC0004ED42C3FFFC188FBD88F8EC00A2
S111900AC3000A188FBD8935EC00C3000A1894
S10F90188FBD88F818CE940BBD891EBDD6
S11190248D862C23EC348A00CA08ED34C62D48
S1109032E731EC00C3000A188FBD88F8BDBB
S110903F8D11EC00C3000A188FBD8935CCDB
S111904C000A3736EC00C3000A188FBD88F8FE
S111905A183C183C1830BD8935EC29BD87E65A
S1119068BD86E1062039EC42C30002ED42C38E
S1119076FFFE188F18EC00ED0E2C14EC348A5B
S111908400CA08ED34C62DE731EC0E405082D0
S111909200ED0ECC000A3736EC0E3736EC2912
S11190A0BD875818381838EC00C30010ED2BAB
S11190AE7E925EEC348400C4021A8300002714
S11190BC1BEC42C30004ED42C3FFFC188FBD41
S11190CA88F8EC00C3000A188FBD8935201108
S11190D8EC42C30002ED42C3FFFE188F18ECF9
S11190E600ED0E1AEE4018E600C1752645ECAA
S11190F4348400C4021A8300002724CC000A2E
S11191023736EC00C3000A188FBD88F8183CFD
S1109110183C1830BD8935EC29BD87E6BD3B
S111911D86E1067E9216CC000A3736EC0E3739
S111912B36EC29BD8758183818387E92161A6B
S1119139EE4018E600C16F27037E91A7EC34C8
S11191478400C4011A8300002711EC29ED06F0
S1119155C30001ED291AEE06C63018E700EC3F
S1119163348400C4021A8300002724CC0008C0
S11191713736EC00C3000A188FBD88F8183C8E
S110917F183C1830BD8935EC29BD87E6BDCC
S111918C86E1067E9216CC00083736EC0E37CC
S111919A36EC29BD8758183818387E9216EC2A
S11191A8348400C4011A8300002722EC29ED50
S11191B606C30001ED291AEE06C63018E700C4
S11191C4EC29ED04C30001ED291AEE04C6786F
S11191D218E700EC348400C4021A830000275E
S11191E023CC00103736EC00C3000A188FBDF4
S11191EE88F8183C183C1830BD8935EC29BDB2
S11191FC87E6BD86E1062012CC00103736EC63
S111920A0E3736EC29BD875818381838EC009A
S1119218C30010ED2B203FEC42C30002ED42D8
S1119226C3FFFE188F18EC00ED0E3736EC3A3D
S11192341AEE3E18AD001838EC2FC30001ED01
S11192422F7E93B0EC42C30002ED42C3FFFE48
S1119250188F18EC00ED2B2605CC93F9ED2BAE
S111925EEC2BBD94AEED02EC32A302ED32EC2B
S111926C2D2607EC2BBD94AEED2DEC348400C2
S111927AC4081A8300002707EC32830001EDBC
S111928832EC348400C4101A83000026037EE6
S111929692F3EC348400C4081A830000271AF3
S11192A4E6314F5D2A01433736EC3A1AEE3EAE
S11192B218AD001838EC2FC30001ED2FEC347A
S11192C08400C4041A83000027037E936A20EE
S11192CE1DCC00303736EC3A1AEE3E18AD00D7
S11192DC1838EC2FC30001ED2FEC3283000193
S11192EAED32EC322EDF7E936AEC348400C445
S11192F8041A8300002623201DCC00203736E4
S1109306EC3A1AEE3E18AD001838EC2FC3F7
S11193130001ED2FEC32830001ED32EC322E1E
S1119321DFEC348400C4081A830000273CE605
S111932F314F5D2A01433736EC3A1AEE3E18F0
S111933DAD0018382027EC2BED06C30001ED1F
S111934B2B1AEE0618E6004F5D2A0143373652
S1109359EC3A1AEE3E18AD001838EC2FC3A4
S11193660001ED2FEC2DED04830001ED2DEC44
S11193740426CCEC348400C4041A83000027C1
S11193822D201DCC00203736EC3A1AEE3E1892
S1119390AD001838EC2FC30001ED2FEC328332
S111939E0001ED32EC322EDF2008CC93CEED30
S11193AC2B7E925EEC40C30001ED401AEE40B1
S11193BA186D0027037E8E07EC2F8FC300383A
S11193C88F35381838393C696E7465676572E4
S11193D6206F6E6C79207072696E742C207595
S11193E47365202D6C66703F3F20746F2072FD
S11193F2656C696E6B3E00286E756C6C2070A5
S110940074722070617373656429000000AC
S105940D000059
S111940F3C30188FEE04183CE600270818E7DE
S110941D0008180820F418E700323338392D
S111942A37363C3C30EF00E6094F5D2A014323
S1119438BD871108083538183839BD86BA4684
S1109446CC00023736EC00C300083736CCEA
S11194530000EC00C30006BD948418381838DD
S1119461ED043736EC083736CC942A3736CC77
S110946F0000BD8DFBBD86E106ED028FC33C
S10B947C00068F353818383959
S111948437363C3C30EF00EC04C300021AA360
S1119492082607EC04C300062004EC0AE308D5
S10A94A008083538183839BB
S10A94A7CC0030BD87403901
S11194AEBD86BA46CC0000ED042007EC04C3D2
S11194BC0001ED04EC08ED02C30001ED081AF6
S11194CAEE02186D0026E8EC048FC300068F36
S10894D8353818383995
S11194DDBD86BA4A2007EC0CC30001ED0C1A40
S11194EBEE0C18E6004F5D2A0143BD97721A7D
S11194F983000026E5CC0000ED061AEE0C18E8
S1119507E600C12D260ECC0001ED06EC0CC3CF
S11195150001ED0C20111AEE0C18E600C12B1B
S11195232607EC0CC30001ED0CCC0000ED0893
S1119531202AEC0CED04C30001ED0CCC000A62
S111953F1AEE08BD86691AEE04373618E600E7
S111954D4F5D2A0143ED023233E30283003006
S111955BED081AEE0C18E6004F5D2A0143BD20
S111956996E11A83000026C2EC062708EC08DF
S1119577405082002002EC088FC3000A8F359A
S1079585381838391D
S11195890020202020202020202030303030F0
S11195973020202020202020202020202020F2
S11195A5202020202090404040404040404084
S11195B3404040404040400C0C0C0C0C0C0C92
S11195C10C0C0C404040404040400909090990
S11195CF09090101010101010101010101016C
S11195DD0101010101010101404040404040F4
S11195EB0A0A0A0A0A0A020202020202020222
S11195F90202020202020202020202024040C8
S110960740402000000000000000000000B2
S1119614000000000000000000000000000044
S1119622000000000000000000000000000036
S1119630000000000000000000000000000028
S111963E00000000000000000000000000001A
S111964C00000000000000000000000000000C
S111965A0000000000000000000000000000FE
S11196680000000000000000000000000000F0
S11196760000000000000000000000000000E2
S111968400000000000037363C3C30EF00ECE4
S111969204C3958A188F18E6004F8400C4079D
S11196A00808353818383937363C3C30EF00AE
S11196AEEC04C3958A188F18E6004F8400C49C
S11196BC030808353818383937363C3C30EF8F
S11196CA00EC04C3958A188F18E6004F840044
S11196D8C4200808353818383937363C3C3081
S11196E6EF00EC04C3958A188F18E6004F8439
S11196F400C4040808353818383937363C3CB1
S111970230EF00EC04C3958A188F18E6004F70
S11197108400C4470808353818383937363C09
S111971E3C30EF00EC04C3958A188F18E60067
S111972C4F8400C4020808353818383937361F
S111973A3C3C30EF00EC04C3958A188F18E60F
S1119748004F8400C4570808353818383937E4
S1119756363C3C30EF00EC04C3958A188F18A3
S1119764E6004F8400C4400808353818383930
S111977237363C3C30EF00EC04C3958A188F68
S111978018E6004F8400C41008083538183865
S111978E3937363C3C30EF00EC04C3958A18A2
S111979C8F18E6004F8400C401080835381801
S11197AA383937363C3C30EF00EC04C3958A66
S11197B8188F18E6004F8400C40808083538DE
S11097C618383937363C3C30EF00EC04BD58
S11197D3978F1A830000270AEC04830041C319
S11197E100612002EC040808353818383937C6
S11097EF363C3C30EF00EC04BD971B1A83A0
S11197FC0000270AEC04830061C30041200230
S10C980AEC04080835381838395B
S11198133B3B3B3B3B3B3B3B3B3B3B3B3B3B09
S10598213B3BCB
S1059AE7FFD6A4
S1109823BD86BA44CC9ABABD94422023CC31
S11198300001BD81443736CC9AA1BD94421884
S111983E3818CE1000181C0080EC0C3736ECE5
S110984C0ABD98A41838CC0001BD8144C3A6
S1119859000AED02EC061AA30222CB2023CC57
S11198670001BD81443736CC9AA1BD9442184D
S11198753818CE1000181D0080EC0C3736ECAD
S11098830ABD98A41838CC0001BD814483AF
S1119890000AED02EC061AA30225CB08080814
S111989E08353818383937363C3C30EF00CCEA
S11198AC9A91BD944218CE1022181C00401848
S11198BACE1020181C0040EC04FD9B0AEC08A4
S11198C8FD9B080808353818383918CE1022D0
S11198D6181D004018CE1020181C008018CE5B
S11198E4100B181C004039FC1018F39B0AFDF1
S11198F2101818CE1023181D00BF3B1B5B324C
S11199004A04001B5B313B314800BD86BA109F
S111990EEC00C3000A18CE98FD3C8FCC000676
S111991CBD86A238EC00C3000318CE99033CAC
S111992A8FCC0007BD86A23818CE1026181C5C
S11199380080BD813BBD8040BD83810EEC00EC
S1119946C3000A3736CC9A8EBD94421838EC12
S111995400C300033736CC9A8EBD94421838F7
S10D9962CC9A3EBD9442CC9A16BD87
S10E996C94422038CC99EDBD9442BD1C
S10C9977856FFD9B02CC99CEBD65
S10C99809442BD856FFD9B04CCEB
S10C998999B2BD9442BD856FFD45
S11099929B06FC9B023736FC9B043736FC19
S110999F9B06BD98231838183820C68FC3C6
S10999AC00108F3538396C
S11199B2456E7465722074686520646573697F
S11199C072656420706F736974696F6E0A00BB
S11199CE456E746572206520636C6F636B7365
S11199DC20666F722064757479206379636C61
S11199EA650A00456E746572206E756D6265C7
S11199F872206F66206520636C6F636B7320B2
S1119A06666F722074686520706572696F6403
S1119A140A00504E45554D41544943204359D4
S1119A224C494E44455220444941474E4F534F
S1119A305449432050524F4752414D0A0A00F8
S1119A3E095469746C653A090976616C7665A1
S1119A4C2E630A0950726F6772616D6D657248
S1119A5A3A0953636F7474204E6F72746D6119
S1119A686E0A09446174653A09094A616E7513
S1119A766172792C20323030300A0956657244
S1119A8473696F6E0909310A0A0025730059CF
S1119A926F752772652061742050574D2E0A9F
S1119AA00054686520616E616C6F672076610A
S1119AAE6C75652069733A0925640A00596FC6
S1119ABC75277265202061742074686520622D
S1119ACA6567696E6E696E67206F662076614F
S1119AD86C76655F706F736974696F6E2E0A29
S1049AE6007B
S90380007C
